:020000040000FA
:020000007E2858
:080008004F288C0081018316D2
:100010000313C030810508008C008101831603138F
:10002000C030810501308104831203130B110B1DB5
:1000300017288C0B162808009400051008308C0037
:100040002D2014180514141C0510940C2D208C0B55
:10005000212805142D202D2008001D308D00332867
:1000600008308D0033288D0B332808009501732844
:1000700009301C2045301C2063301C2068301C20B7
:100080006F301C203A301C2009301C2015081C2021
:100090000D301C200A301C2013100B1608008B1387
:1000A0008B1B4F289600030E970083010A089800C7
:1000B0008A018313040899008B185F2875280B1296
:1000C00030200618362808308C002D200618951789
:1000D000061C95130C0B950C8C0B65282D20061C0B
:1000E0003628131474280B168B101908840018086E
:1000F0008A00170E8300960E160E09008B018316D8
:1001000003130510061401138312031305148B1037
:100110000B168B1793010D301C200A301C20523017
:100120001C2053301C2032301C2033301C20323035
:100130001C2020301C2054301C2065301C207330C3
:100140001C2074301C2020301C2049301C206E30B4
:100150001C2074301C2065301C2072301C2066303E
:100160001C2061301C2063301C2065301C203A307C
:100170001C2020301C2050301C2049301C204330D3
:100180001C2031301C2036301C2046301C203830DA
:100190001C2034301C2020301C2063301C206F3089
:1001A0001C206E301C206E301C2065301C206330FB
:1001B0001C2074301C2065301C2064301C202E3024
:1001C0001C202E301C202E301C200D301C200A300C
:0C01D0001C200A301C2013183820EB28DB
:02400E00F13F80
:00000001FF
